:1000000058C0EDC171C070C06FC06EC06DC06CC013
:100010006BC06AC069C068C067C066C065C064C0A4
:1000200063C062C061C00403090422037700770043
:1000300077002E0072006500630075007200730087
:1000400069006F006E002E006A00700010035500FA
:10005000530042002D003200330032001201100123
:1000600002000008C016E1050001010200010902BA
:100070004300020100803209040000010202010075
:1000800005240010010424020205240600010524B1
:10009000010301070583030800FF09040100020AA8
:1000A00000000007050102080000070581020800A2
:1000B000000011241FBECFE5D4E0DEBFCDBF10E0AD
:1000C000A0E6B0E0EAE4FAE002C005900D92AC369A
:1000D000B107D9F712E0ACE6B0E001C01D92A4343C
:1000E000B107E1F7FAD3AFC48BCF85B7826085BF84
:1000F0008BB780648BBF8BE4809381008093AC00CE
:100100008AE5809380008093AB0008951F93CF937E
:10011000DF93DC01162FEA01888184FF05C0898105
:1001200098E88927898302C08AE58883AE014E5FFB
:100130005F4F212FFA018D91819321501216DCF32C
:10014000CA01612F48D11C5F1883DF91CF911F91A5
:1001500008954BEA50E0DADF089540E850E0D6DF3A
:1001600008951F93CF93DF9360919100635067FDD3
:10017000B3C080918E00CCE0D0E0C81BD109CB5633
:10018000DF4F80918D00803118F4CE018AD39EC05C
:100190008D3209F08BC0683009F098C083EC8093F1
:1001A00075008AE58093600010926C0088818076EB
:1001B00021F0CE0136D3282F66C09A8110927E009E
:1001C0008981882321F410927F0022E055C0853078
:1001D00019F4909392004FC08630B9F58B8181302D
:1001E00041F48CE590E09093900080938F0022E1A1
:1001F00028C0823021F4CE01FFD2282F22C08330C4
:10020000F9F48A81882341F486E290E0909390008B
:1002100080938F0024E015C0813041F48AE290E0A1
:100220009093900080938F0022E20BC0823041F4C3
:100230008CE490E09093900080938F0020E101C0C7
:1002400020E080E480936C001EC0883021F421E01F
:1002500084E990E013C0893019F4909394000BC0A6
:100260008A3011F421E008C08B3029F48BE48093AC
:1002700081008093AC0020E08EE790E090939000A6
:1002800080938F0009C02F3F39F4888187FD2E812C
:1002900080E880936C0006C08F81882319F48E81DA
:1002A000821708F0822F8093610010C080916C004B
:1002B00087FF0CC0CE016ED38F3F21F48EE1809377
:1002C000600004C0882311F01092610080919100B9
:1002D000181614F4109291008091600084FF58C0A9
:1002E000809161008F3F09F453C0182F893008F0C6
:1002F00018E0811B809361008091750098E8892740
:1003000080937500112391F180916C0087FF08C0E4
:1003100086E790E0612FADD2182F893098F526C07E
:1003200020918F003091900086FF0DC0A6E7B0E0CD
:1003300080E090E0F901E80FF91FE491ED93019658
:100340001817C1F708C0912FD901E6E7F0E08D91A9
:1003500081939150E1F71150812F90E01F5F01963A
:10036000820F931F9093900080938F0086E790E018
:10037000612F31D0612F6C5F6C3041F08FEF809333
:10038000610004C08FEF809361006EE160936000B4
:1003900094E180B38C7031F49150D9F710929200AF
:1003A00010928C00DF91CF911F910895A82FB92F43
:1003B00080E090E041E050EA609530E009C02D9186
:1003C00082279795879510F084279527305EC8F38C
:1003D0006F5FA8F30895EADF8D939D930895CF93FF
:1003E000CFB7CF93C395839BE9F7839B09C0839BCA
:1003F00007C0839B05C0839B03C0839B01C0A6C02D
:10040000DF93C0918E00DD27CB56DF4F839B02C068
:10041000DF91EBCF2F930F931F9300B32FEF03FBCD
:1004200020F94F933F9310B34FEF012703FB21F9BE
:100430003BE031C04E7F012F10B3216028C0102F48
:100440004D7F2260000000B329C04B7F2460012F44
:10045000000010B32BC010B3477F28602AC04F7E26
:1004600000B320612CC04F7D10B320622FC04F7BA2
:1004700000B3206432C0422700B349934FEF00001D
:10048000102713FB20F910B31C70C9F1297F91F2DA
:10049000012703FB21F900B3237F89F2315058F182
:1004A000102713FB22F910B3277E79F2012703FBF3
:1004B00023F92F7C81F200B3102713FB24F92F7945
:1004C00071F200C010B3012703FB25F92F7359F215
:1004D00000C000B3102713FB26F9223040F200C001
:1004E00010B3012703FB27F9243028F64F77206843
:1004F00010B30000F9CF10E41ABF00271CC03B5016
:100500003195C31BD04010E41ABF0881033C11F1A0
:100510000B3401F120918C001981110F1213EDCFD2
:100520004A81441F093659F10D3211F0013E29F775
:100530004F7009F0042F009393003F914F911F914A
:100540000F912F91DF91CAB7C6FD4CCFCF91CFBF8E
:10055000CF91189520919300222379F31091910067
:100560001123C1F53430C2F13093910020938D00F6
:1005700010918E003BE0311B30938E002DC0009116
:10058000910001303CF50AE54F7049F4309160006C
:1005900034FD24C000936000C5E7D0E023C04330A1
:1005A00049F03091800034FD19C000938000C1E80B
:1005B000D0E018C03091AB0034FD10C00093AB0008
:1005C000CCEAD0E00FC02795A8F45150A9F4220F2F
:1005D0000000F9CF4AE503C042ED01C0432FC4E15A
:1005E000D0E032E011B31C60939A11BB02B320E457
:1005F0001CE05F93012756E002BB279520F4515081
:1006000021F4220FF9CF012756E000003B5A02BB2C
:10061000D0F2279528F4515029F4220F0000F9CF89
:10062000012756E0279502BB20F4515021F4220FF8
:10063000F9CF012756E02991332302BB21F6037F2E
:1006400010919200110FC651D04002BB11F01093CF
:100650008C0010E41ABF086011B3137F402F437F52
:100660005F9100C000C002BB11BB42BB66CFBF920E
:10067000CF92DF92EF92FF920F931F936B017C0159
:10068000B42E122F9695879577956795605A7C4181
:10069000894E9F4FA7019601B4D121503040404070
:1006A0005040599A1AB881E0B81611F440EB04C0D2
:1006B0004B2D4295407F4068802F90E00597880F32
:1006C000991F1695110F110F110F182B412B40BDBB
:1006D00029B930BD88E18AB984BB8FEF85BB1F91F2
:1006E0000F91FF90EF90DF90CF90BF9008950F9300
:1006F0001F9330914102909142020FC0E92FF0E028
:10070000E05CFE4F80818CB99F5F8091910087FFF4
:1007100007C0293028F010929100292F231B01C017
:100720002F5F5D9B0BC0391739F4309342029091D3
:100730004002E0913F0115C09D99E0CF90934202A5
:10074000F6CF391751F08BB12CB18C7171F4F0E008
:10075000E954FF4F2083E32F04C0E0933F01AC989E
:1007600008C0EF5F3E2F3F77E1505F99EACFE093FB
:100770003F018091800084FF3CC060913F01691778
:1007800021F4809143028823A1F1162F191B1F77B2
:10079000193008F018E0012F090F07FF10C00F777C
:1007A000A7EBB0E0202F30E02A0F3B1F05C0FD0172
:1007B000E058FF4F8D918083A217B307C1F7892FAF
:1007C00090E089549F4F612FC8DC009340021123B1
:1007D00061F0AC9A183049F490E080913F018013A9
:1007E00091E081E09827892F02C080E090E080931B
:1007F00043021F910F910895FC018381813049F4D8
:100800008CE590E09093900080938F0080915C0045
:1008100008958EE690E09093900080938F0083E49B
:100820000895FC012081822F8076803201F591812C
:10083000892F8052823010F48FEF0895923281F424
:1008400085B392819170990F990F990F877F982B9B
:1008500095BB80916D00882319F482E080936D0030
:1008600027FD05C081E08093430280E0089580E089
:100870000895FC01809171008083809172008183D2
:1008800080917300828380917400838380916E00D5
:10089000848380916F00858380917000868387E0D8
:1008A0000895DC01909142020CC02E2F2F5F291772
:1008B00039F0F0E0E05CFE4F8D918083209341029F
:1008C0006150E0914102662381F791509E1B99305F
:1008D00018F48FEF8093910008950F932EE088E134
:1008E00090E00FB6F894A89581BD0FBE21BD83EFAF
:1008F00082BB8CE081BBA89584EC99E02CE231E0CE
:10090000F9013197F1F70197D9F711BA80E895E22B
:10091000A0E0B0E08093710090937200A093730008
:10092000B093740010926E0010926F0088E0809374
:10093000700060E875E280E090E040E020E008E0D0
:1009400096DE1092420210923F01109240021092E5
:100950004102CBDB10926D00109243027894A8956F
:1009600000DCC5DE90916D009923C9F38091AB0046
:1009700084FFF5CF923021F482E690E068E003C076
:100980008AE690E062E0E5DB80916D008150809323
:100990006D00E5CF0F93FC01808180937100818110
:1009A00080937200828180937300838180937400AE
:1009B000948190936E00858180936F0006810093EF
:1009C0007000833010F010926F00913011F410928B
:1009D0006E0060917100709172008091730090912F
:1009E000740040916F0020916E0041DE109242022F
:1009F00010923F01109240021092410281E00F914B
:100A00000895A1E21A2EAA1BBB1BFD010DC0AA1F4F
:100A1000BB1FEE1FFF1FA217B307E407F50720F067
:100A2000A21BB30BE40BF50B661F771F881F991FE2
:100A30001A9469F760957095809590959B01AC012B
:0A0A4000BD01CF010895F894FFCF27
:0C0A4A005AFFA120000000000200030081
:00000001FF
